S020000064656D6F70726F675F6F6C696D6578696E6F5F73746D33322E737265635C
S3150800800000500020C58C0008158D0008158D000845
S31508008010158D0008158D0008158D00080000000054
S31508008020000000000000000000000000158D000898
S31508008030158D000800000000158D00084D8D0008FC
S31508008040158D0008158D0008158D0008158D00087A
S31508008050158D0008158D0008158D0008158D00086A
S31508008060158D0008158D0008158D0008158D00085A
S31508008070158D0008158D0008158D0008158D00084A
S31508008080158D0008158D0008158D0008158D00083A
S31508008090158D0008158D0008158D0008158D00082A
S315080080A0158D0008158D0008158D0008158D00081A
S315080080B0158D0008158D0008158D0008158D00080A
S315080080C0158D0008158D0008158D0008158D0008FA
S315080080D0158D0008158D0008158D0008158D0008EA
S315080080E0158D0008158D0008158D00080000000084
S315080080F00000000000000000000000000000000072
S3150800810000000000000000005FF808F1EE11AA5513
S3150800811010B5054C237833B9044B13B10448AFF3B3
S3150800812000800123237010BD0C0000200000000011
S31508008130A08D000808B5034B1BB103490348AFF3EC
S31508008140008008BD0000000010000020A08D000877
S315080081507047704708B500222021024800F0DAF976
S3150800816008BD00BF0008014010B500F0EBFD0E4B3E
S315080081701B68C31AB3F5FA7F0CD304460B4B1B785E
S315080081804BB90122094B1A702021094800F0C2F99F
S31508008190054B1C6010BD0022044B1A7020210448B0
S315080081A000F0B8F9F4E700BF2C00002028000020F2
S315080081B00008014010B504460E4B18784FF47A7340
S315080081C0B3FBF0F30C4A1068B0FBF3F000F080F84C
S315080081D068B90F2C01D9012010BD002221464FF0A5
S315080081E0FF3000F043F8054B1C60002010BD01204D
S315080081F010BD00BF00000020080000200400002079
S3150800820008B5074A136843F010031360032000F00B
S315080082101BF80020FFF7CEFF00F0ECFC002008BD9D
S3150800822000200240034A1168034B1B780B44136075
S31508008230704700BF3000002000000020014B18687E
S31508008240704700BF30000020074AD36823F4E06374
S315080082501B041B0C000200F4E060184340F0BF60EA
S3150800826040F40030D060704700ED00E030B4164BA3
S31508008270DB68C3F30223C3F10704042C28BF0424D4
S315080082801D1D062D17D9033B012505FA04F4013CEB
S315080082902140994005FA03F3013B1340194300288E
S315080082A00BDB0901C9B200F1604000F5614080F8B6
S315080082B0001330BC70470023E6E700F00F00090101
S315080082C0C9B2024B1954F4E700ED00E014ED00E0E2
S315080082D00138B0F1807F0AD2064B5860F021064A71
S315080082E082F823100020986007221A607047012040
S315080082F0704700BF10E000E000ED00E0042805D05C
S31508008300054A136823F0040313607047024A13688A
S3150800831043F004031360704710E000E0704708B5A7
S31508008320FFF7FCFF08BD0000F0B583B00026344611
S3150800833071E0002D00F0A180012D00D1CE68FF2B41
S3150800834000F2AF808646FF2B00F2AE80A500DEF86D
S3150800835000200F27AF4022EA070206FA05F52A434E
S31508008360CEF800204A6812F0805F53D0634A9569B8
S3150800837045F001059561926902F001020192019AA0
S31508008380A508AF1C5E4A52F8272004F00307BF0071
S315080083904FF00F0E0EFA07FE22EA0E02DFF870E122
S315080083A0704500F088800EF5806E704500F0868076
S315080083B00EF5806E704500F084800EF5806E70456F
S315080083C076D04FF0040E0EFA07F73A4302354C4FB3
S315080083D047F825204A6812F4803F75D0494D2A6827
S315080083E01A432A604A6812F4003F73D0454D6A68FA
S315080083F01A436A604A6812F4801F71D0414DAA6810
S315080084001A43AA604A6812F4001F6FD03D4DEA6805
S315080084101343EB6001340F2C6ED80122A2400B687F
S3150800842013409A42F6D14D68122D30D00BD8022D42
S315080084302AD07FF67EAF032D2FD0112D7FF47FAF84
S31508008440CE6804367BE7304FBD4216D00CD92F4F85
S31508008450BD4212D007F58037BD420ED0A7F580176A
S31508008460BD427FF46CAF08E0A7F58017BD4204D083
S3150800847007F58037BD427FF462AF8D687DB1012D67
S3150800848008D0426108265AE7CE68083657E7CE680C
S315080084900C3654E70261082651E700264FE7042602
S315080084A04DE700F1040E4EE7A4F10805AD004EE7CE
S315080084B04FF0030E87E74FF0000E84E74FF0010EEA
S315080084C081E74FF0020E7EE70E4D2A6822EA030284
S315080084D02A6087E70B4D6A6822EA03026A6089E721
S315080084E0084DAA6822EA0302AA608BE7054DEA68E6
S315080084F022EA0303EB608DE703B0F0BD00100240EB
S315080085000000014000040140000021100000311065
S315080085100008014012B909040161704701617047FA
S3150800852082B0084B1B68084AA2FB03235B0A00FBC0
S3150800853003F0019000BF019B5A1E0192002BF9D14E
S3150800854002B0704708000020D34D621070B582B0A3
S315080085500446036813F0010F3DD0AC4B5B6803F08B
S315080085600C03042B2ED0A94B5B6803F00C03082BD5
S3150800857023D06368B3F5803F51D0002B55D103F162
S31508008580804303F504331A6822F480321A601A68A5
S3150800859022F480221A606368002B60D0FFF74EFE33
S315080085A005469A4B1B6813F4003F14D1FFF746FEA5
S315080085B0401B6428F5D90320AFE1944B5B6813F49C
S315080085C0803FD6D0914B1B6813F4003F03D06368F5
S315080085D0002B00F09F81236813F0020F65D08B4BA8
S315080085E05B6813F00C0F4ED0884B5B6803F00C03E6
S315080085F0082B43D02369002B79D00122844B1A60BB
S31508008600FFF71CFE0546814B1B6813F0020F65D168
S31508008610FFF714FE401B0228F5D903207DE17B4AAB
S31508008620136843F480331360B5E7B3F5A02F09D078
S31508008630764B1A6822F480321A601A6822F480226D
S315080086401A60A8E703F18043A3F53C331A6842F49D
S3150800865080221A601A6842F480321A609BE7FFF794
S31508008660EDFD0546694B1B6813F4003FB3D0FFF7D1
S31508008670E5FD401B6428F5D903204EE1634B5B6892
S3150800868013F4803FB6D1614B1B6813F0020F04D078
S315080086902369012B01D001203FE15C4A136823F0CE
S315080086A0F803616943EAC1031360236813F0080FEE
S315080086B032D0A369002B6ED00122564B1A60FFF701
S315080086C0BDFD0546514B5B6A13F0020F21D1FFF73A
S315080086D0B5FD401B0228F5D903201EE14B4A136855
S315080086E023F0F803616943EAC1031360DDE700225A
S315080086F0474B1A60FFF7A2FD0546444B1B6813F06B
S31508008700020FD2D0FFF79AFD401B0228F5D90320A5
S3150800871003E10120FFF704FF236813F0040F00F0BC
S3150800872099803A4BDB6913F0805F46D1374BDA699B
S3150800873042F08052DA61DB6903F080530193019BB2
S315080087400125354B1B6813F4807F38D0E368012B6D
S3150800875049D0002B4DD103F1804303F504331A6A3F
S3150800876022F001021A621A6A22F004021A62E36807
S31508008770002B5DD0FFF762FD0646244B1B6A13F0FB
S31508008780020F66D1FFF75AFD801B41F288339842E3
S31508008790F3D90320C1E000221E4B1A60FFF74EFDF5
S315080087A005461A4B5B6A13F0020FB5D0FFF746FD74
S315080087B0401B0228F5D90320AFE00025C1E7164A79
S315080087C0136843F480731360FFF738FD0646124BAF
S315080087D01B6813F4807FB9D1FFF730FD801B64282E
S315080087E0F5D9032099E0094A136A43F00103136295
S315080087F0BDE7052B12D0054B1A6A22F001021A6250
S315080088001A6A22F004021A62B1E700BF0010024099
S31508008810000042428004424200700040414B1A6AFE
S3150800882042F004021A621A6A42F001021A629EE7CC
S31508008830FFF704FD06463B4B1B6A13F0020F08D0F0
S31508008840FFF7FCFC801B41F288339842F3D90320DA
S3150800885063E0E5B9E369002B5ED0324A526802F05C
S315080088600C02082A5BD0022B17D000222E4B1A6066
S31508008870FFF7E4FC04462B4B1B6813F0007F47D038
S31508008880FFF7DCFC001B0228F5D9032045E0254A42
S31508008890D36923F08053D361DCE70022224B1A60A8
S315080088A0FFF7CCFC05461F4B1B6813F0007F06D06C
S315080088B0FFF7C4FC401B0228F5D903202DE0236AE4
S315080088C0B3F5803F1AD017494B6823F47413226A0C
S315080088D0606A024313434B600122134B1A60FFF789
S315080088E0ADFC04460F4B1B6813F0007F0ED1FFF753
S315080088F0A5FC001B0228F5D903200EE0094A536897
S3150800890023F40033A1680B435360DCE7002004E03E
S31508008910002002E0012000E0002002B070BD012026
S31508008920FBE700BF001002406000424210B586B067
S31508008930154C94E80F000DF1180E0EE90F00238A66
S31508008940ADF80430114B5B6803F00C02082A18D105
S31508008950C3F38342724412F8102C13F4803F03D1F8
S315080089600B4800FB02F00DE0084B5B68C3F340437D
S31508008970734413F8143C074800FB02F0B0FBF3F00D
S3150800898000E0044806B010BDB88D0008001002408B
S3150800899000093D0000127A00594B1B6803F00703D3
S315080089A08B420CD2564A136823F007030B43136015
S315080089B0136803F00703994201D00120704770B588
S315080089C0036813F0020F06D04E4A536823F0F003EB
S315080089D08468234353600D460446036813F0010F69
S315080089E052D04368012B23D0022B28D0454A12685F
S315080089F012F0020F00F0828042494A6822F0030210
S31508008A0013434B60FFF71AFC06466368012B1DD01B
S31508008A10022B2AD03B4B5B6813F00C0F34D0FFF7C0
S31508008A200DFC801B41F288339842F3D9032070BDB0
S31508008A30344A126812F4003FDED1012070BD314A73
S31508008A40126812F0007FD7D1012070BD2D4B5B68EC
S31508008A5003F00C03042B17D0FFF7F0FB801B41F241
S31508008A6088339842F2D9032070BD264B5B6803F021
S31508008A700C03082B08D0FFF7E1FB801B41F2883373
S31508008A809842F2D9032070BD1D4B1B6803F00703FB
S31508008A909D420CD21A4A136823F007032B4313602E
S31508008AA0136803F007039D4201D0012070BD2368B7
S31508008AB013F0040F06D0134A536823F4E063E16801
S31508008AC00B435360236813F0080F07D00D4A536809
S31508008AD023F46053216943EAC1035360FFF726FF75
S31508008AE0084B5B68C3F30313074AD35CD840074BAC
S31508008AF018600020FFF75EFB002070BD012070BDE6
S31508008B000020024000100240CC8D0008080000201A
S31508008B10014B1868704700BF080000200F4B1A6801
S31508008B2042F001021A6059680D4A0A405A601A68EA
S31508008B3022F0847222F480321A601A6822F48022A3
S31508008B401A605A6822F4FE025A604FF41F029A60AD
S31508008B504FF00062034B9A60704700BF0010024056
S31508008B600000FFF800ED00E0014B024A9A607047EA
S31508008B7000ED00E00080000800B591B001220692E1
S31508008B804FF480330793002108910A9202220D922E
S31508008B900E934FF4E0130F9306A8FFF7D7FC00B126
S31508008BA0FEE70F23019302210291002303934FF45A
S31508008BB080620492059301A8FFF7EEFE00B1FEE776
S31508008BC011B05DF804FB08B5FFF7CEFFFFF718FBF9
S31508008BD0FFF7D2FF00F0A0F8FFF7BCFA08BD08B50A
S31508008BE0FFF7F1FFFFF7B4FAFFF7BEFAFFF7B1FA9E
S31508008BF0FAE7000000B589B0304B9A6942F00102E5
S31508008C009A619A6902F001020092009ADA6942F0C2
S31508008C108052DA61DA6902F080520192019A9A6901
S31508008C2042F004029A619A6902F004020292029AD8
S31508008C309A6942F008029A619B6903F00803039354
S31508008C40039B0320FFF700FB002211466FF00B0081
S31508008C50FFF70CFB002211466FF00A00FFF706FB30
S31508008C60002211466FF00900FFF700FB00221146AB
S31508008C706FF00400FFF7FAFA002211466FF00300BE
S31508008C80FFF7F4FA002211466FF00100FFF7EEFA3B
S31508008C90002211464FF0FF30FFF7E8FA202304932D
S31508008CA001230593002306930223079304A9044886
S31508008CB0FFF73AFB09B05DF804FB00BF001002405D
S31508008CC000080140DFF834D0002103E00C4B5B5864
S31508008CD0435004310B480C4B42189A42F6D30B4AC0
S31508008CE002E0002342F8043B094B9A42F9D3FFF706
S31508008CF015FF00F031F8FFF772FF704700500020AB
S31508008D00E48D0008000000200C0000200C00002064
S31508008D1034000020FEE7000008B5FFF7F9FE084B0F
S31508008D20A3FB00308009FFF7D3FA0420FFF7E6FA21
S31508008D30002211464FF0FF30FFF798FA08BD00BF32
S31508008D40D34D621008B5FFF779FA08BD08B5FFF7E5
S31508008D5069FAFFF7E4FA08BD70B500250C4E0D4C0C
S31508008D60A41BA410A54209D100F01AF800250A4E42
S31508008D700A4CA41BA410A54205D170BD56F825308F
S31508008D8098470135EEE756F8253098470135F2E75A
S31508008D90DC8D0008DC8D0008DC8D0008E08D0008FD
S31508008DA0F8B500BFF8BC08BC9E467047F8B500BFCA
S30D08008DB0F8BC08BC9E4670479A
S31508008DB802030405060708090A0B0C0D0E0F101006
S31508008DC80102000000000000000000000102030480
S30908008DD8060708096B
S30908008DDC35810008C7
S30908008DE011810008E7
S31108008DE4010000001000000000A24A0474
S70508008CC5A1
